:100000000C94F3000C940E010C940E010C940E0150
:100010000C940E010C940E010C94DC160C940E0141
:100020000C940E010C940E010C94A9160C946A16F3
:100030000C9462110C940E010C940E010C940E01A0
:100040000C940E010C943B040C940E010C941F10A4
:100050000C9476100C940E010C940E010C940E016D
:100060000C940E010C940E010C940E010C940E01D4
:100070004570692D4F5344205665722E302E382E10
:10008000322E340000416B7475656C6C65732053BF
:10009000657474696E67000053657474696E6720D7
:1000A000200000486F6568656E73656E736F72201F
:1000B00000004853206D697420536368616C746557
:1000C0007220000048656164696E6720486F6C6447
:1000D0002000004B6F6D706173732000004B6F6DDB
:1000E0007061737320666978200000475053204187
:1000F0006B74697620000041636873656E6B6F7086
:1001000070656C756E67200000447265687261747A
:100110006520626567722E2000004665686C657216
:100120002046433C2D3E4F5344200000556E7465DD
:10013000727370616E6E756E672000004B65696E3C
:10014000652053657474696E672D416E7A656967C1
:1001500065000050432F4254206973742065696E16
:100160006765736368616C746574000055656265EA
:10017000726E65686D65204C65747A746573205382
:10018000657474696E6700004F4E00002D2D2D00C0
:10019000004550492D4D656E750050616C0050430F
:1001A0002F4254004B656E6E756E670052432D42B0
:1001B000657472696562000045786974004F4E008D
:1001C0002D2D0076767D76767A76767E76767776C3
:1001D000767B76767876767C76767976767D7676A8
:1001E0007A76767E760011241FBECFEFD4E0DEBF94
:1001F000CDBF11E0A0E0B1E0EAE6F1E302C0059076
:100200000D92AE34B107D9F713E0AEE4B1E001C00E
:100210001D92AC3AB107E1F70C941B010C9400005D
:1002200080E981BB8FE084BBAC9AAD9A8EE28ABB39
:10023000D99ADD9A08951F93109295011092910119
:1002400010929601A0E0B0E00E94A118802D99279D
:1002500080935501A1E0B0E00E94A118802D99275C
:1002600080930001A2E0B0E00E94A118802D9927A0
:1002700080935601A7E1B0E00E94A118802D992734
:1002800080936D01A8E1B0E00E94A118802D99270C
:10029000809380010E940F160E9410010E942B047F
:1002A00080915501813019F40E940A1002C00E9409
:1002B000FA0F7894A89A0E94C1030E949C040E949D
:1002C000A3088091800185FF02C00E9447130E940D
:1002D000EB08809150018130B1F41092500180916F
:1002E0009501882351F480915501882331F4809140
:1002F0006201813011F40E9418110E9455110E9470
:100300005A110E940B1480915401909195018130F3
:1003100061F4992351F40E940A0E8091800185FFB7
:1003200004C00E94E6120E944F1380915301813055
:10033000B9F580919501882399F5AA9A0E940A0F30
:1003400080916D018823A9F40E9401080E94F106A2
:100350008091800180FF04C00E94D5110E94820913
:100360008091800183FF02C00E949A170E945B095E
:1003700016C080910201823054F00E94AB080E94A6
:10038000D5110E9482090E947F0A0E945B09809118
:100390000201833024F00E9401080E94F106AA980D
:1003A00080914E018130C1F5809195018823A1F59E
:1003B00010924E0180916D01882321F080910201FD
:1003C000833014F00E94320980916A0190916B0190
:1003D000019690936B0180936A0180916A019091DC
:1003E0006B01CC9769F48091680190916901019645
:1003F000909369018093680110926B0110926A01D9
:100400000E94E10A0E94200980915B01813021F461
:100410000E94950B0E94210D10914F01113009F09F
:1004200058CF80919501882309F053CF10924F0146
:100430000E94AB0880918601813019F0823059F416
:1004400006C00E947D0982E08093860104C00E945C
:1004500056091093860180916D01813009F039CFE2
:1004600080919501882309F034CF80916C0181300F
:1004700009F02FCF10926C0180910201813071F050
:1004800082301CF4882339F024CF823081F083300D
:1004900009F01FCF15C00E947D091BCF0E9456098D
:1004A00064E084E00E946D020E949D0412CF0E94CD
:1004B000560964E084E00E946D020E94A30807CF01
:1004C0000E94560964E084E00E946D020E94A30825
:1004D0000E94EB080E943209FCCE482FD99827E0F1
:1004E00030E0DB98000000000000000081E090E0B8
:1004F000022E02C0880F991F0A94E2F7842311F09C
:10050000DA9A01C0DA980000000000000000DB9ACF
:100510000000000000000000215030408FEF2F3F0E
:100520003807F9F627E030E0DB9800000000000013
:10053000000081E090E0022E02C0880F991F0A940B
:10054000E2F7862311F0DA9A01C0DA980000000081
:1005500000000000DB9A00000000000000002150B5
:1005600030408FEF2F3F3807F9F6DB98DA98D99AA9
:10057000089564E084E00E946D026CE080E00E94D7
:100580006D0210925001809150018823E1F36AE0DE
:100590008CE60E946D0260E085E00E946D02089585
:1005A0001F93CF93DF9380914E018823E1F3109244
:1005B0004E010E94CA1010E00DC08091530181309D
:1005C00011F40E940A0F80914E01813019F41092AB
:1005D0004E0111E09091810180E0112309F481E046
:1005E000992311F4882349F7C8E1D0E0882309F45E
:1005F000B1C0809190038093800180918001DE01E1
:10060000082E0E94A91845E850E061E082E00E94AF
:10061000350D48E950E062E082E00E94350D43EA82
:1006200050E064E082E00E94350D42EB50E065E06E
:1006300082E00E94350D44EC50E066E082E00E94CA
:10064000350D43ED50E067E082E00E94350D4DED41
:1006500050E068E082E00E94350D4BEE50E069E02A
:1006600082E00E94350D47EF50E06AE082E00E9490
:10067000350D4CE251E06BE082E00E94350D409177
:100680007E0150917F0162E084E10E94F60C80912E
:10069000800180FF03C048E851E002C04CE851E00F
:1006A00064E084E10E94350D8091800181FF03C0E8
:1006B00048E851E002C04CE851E065E084E10E9466
:1006C000350D8091800182FF03C048E851E002C0EF
:1006D0004CE851E066E084E10E94350D8091800194
:1006E00083FF03C048E851E002C04CE851E067E0F6
:1006F00084E10E94350D8091800184FF03C048E8A9
:1007000051E002C04CE851E068E084E10E94350D00
:100710008091800185FF03C048E851E002C04CE8A9
:1007200051E069E084E10E94350D8091800186FFEF
:1007300003C048E851E002C04CE851E06AE084E1BF
:100740000E94350D4091A00355276BE084E10E9483
:10075000F60C13C045E850E062E082E00E94350DDF
:100760004AE151E065E082E00E94350DDE010E9421
:10077000A118802D992780938001DF91CF911F913F
:1007800008950E94B90210924E0180914E01882373
:10079000E1F340E750E062E087E00E94350D0E94FF
:1007A0009D0410924E0180914E018823E1F3109236
:1007B0004E0180914E018823E1F310924E0164E0D6
:1007C00084E00E946D026CE480E00E946D028091E2
:1007D0005501882319F40E94D0021AC04CE351E05D
:1007E00062E082E00E94350D43E551E064E082E082
:1007F0000E94350D4CE651E066E082E00E94350D26
:10080000A8E1B0E00E94A118802D99278093800173
:1008100080914E018823E1F310924E0180914E01A8
:100820008823E1F310924E0180914E018823E1F379
:1008300010924E0180914E018823E1F310924E01F7
:1008400080914E018823E1F310924E0164E084E030
:100850000E946D02089582E083BF92E49EBD8EE106
:1008600089BF83E087BD86E982BD90938A0080E2DC
:1008700080937D0008951F920F920FB60F9211245E
:100880008F939F93809152018F5F8093520180914B
:100890005201883439F591E0909351011092520140
:1008A0008091A4038F5F8093A4038091A403843676
:1008B00031F41092A40390934E0190934F018091D4
:1008C000A403823311F490934F018091A3038F5FAF
:1008D0008093A3038091A3038A3021F41092A30391
:1008E000909350019F918F910F900FBE0F901F908A
:1008F0001895282F80538A3010F090E005C02033DF
:1009000011F49AE001C0982F822F81548A3110F49B
:10091000922F9653822F81568A3110F4922F9C5336
:100920002D3211F499E403C02E3209F491E4892F99
:10093000992787FD90950895089560E085E00E94CD
:100940006D0263E886E00E946D0260E987E00E9424
:100950006D0260E085E00E946D0264E886E00E941E
:100960006D0261E987E00E946D0260E085E00E940F
:100970006D0265E886E00E946D0262E987E00E94F0
:100980006D0260E085E00E946D0266E886E00E94EC
:100990006D0263E987E00E946D0260E085E00E94DD
:1009A0006D0267E886E00E946D0264E987E00E94BC
:1009B0006D0260E085E00E946D0268E886E00E94BA
:1009C0006D0265E987E00E946D0260E085E00E94AB
:1009D0006D0269E886E00E946D0266E987E00E9488
:1009E0006D0260E085E00E946D026AE886E00E9488
:1009F0006D0267E987E00E946D0260E085E00E9479
:100A00006D0261EA86E00E946D0268E987E00E945B
:100A10006D0260E085E00E946D0262EA86E00E945D
:100A20006D0269E987E00E946D0260E085E00E9446
:100A30006D0263EA86E00E946D026AE987E00E9427
:100A40006D0260E085E00E946D0264EA86E00E942B
:100A50006D026BE987E00E946D0260E085E00E9414
:100A60006D0265EA86E00E946D026CE987E00E94F3
:100A70006D0260E085E00E946D0266EA86E00E94F9
:100A80006D026DE987E00E946D0260E085E00E94E2
:100A90006D0267EA86E00E946D026EE987E00E94BF
:100AA0006D0260E085E00E946D0268EA86E00E94C7
:100AB0006D026FE987E00E946D0260E085E00E94B0
:100AC0006D026FEB86E00E946D0260EA87E00E9493
:100AD0006D0260E085E00E946D0260EC86E00E949D
:100AE0006D0261EA87E00E946D0260E085E00E948D
:100AF0006D0261EC86E00E946D0262EA87E00E946E
:100B00006D0260E085E00E946D0262EC86E00E946A
:100B10006D0263EA87E00E946D0260E085E00E945A
:100B20006D0263EC86E00E946D0264EA87E00E9439
:100B30006D0260E085E00E946D0264EC86E00E9438
:100B40006D0265EA87E00E946D0260E085E00E9428
:100B50006D0265EC86E00E946D0266EA87E00E9405
:100B60006D0260E085E00E946D0266EC86E00E9406
:100B70006D0267EA87E00E946D0260E085E00E94F6
:100B80006D026DED86E00E946D0268EA87E00E94CA
:100B90006D0260E085E00E946D026EED86E00E94CD
:100BA0006D0269EA87E00E946D0260E085E00E94C4
:100BB0006D026FED86E00E946D026AEA87E00E9496
:100BC0006D0260E085E00E946D0260EE86E00E94AA
:100BD0006D026BEA87E00E946D0260E085E00E9492
:100BE0006D0261EE86E00E946D026CEA87E00E9471
:100BF0006D0260E085E00E946D0262EE86E00E9478
:100C00006D026DEA87E00E946D0260E085E00E945F
:100C10006D0263EE86E00E946D026EEA87E00E943C
:100C20006D0260E085E00E946D0264EE86E00E9445
:100C30006D026FEA87E00E946D0260E085E00E942D
:100C40006D026BEF86E00E946D0260EB87E00E9410
:100C50006D0260E085E00E946D026CEF86E00E940C
:100C60006D0261EB87E00E946D0260E085E00E940A
:100C70006D026DEF86E00E946D0262EB87E00E94DC
:100C80006D0260E085E00E946D026EEF86E00E94DA
:100C90006D0263EB87E00E946D0260E085E00E94D8
:100CA0006D026FEF86E00E946D0264EB87E00E94A8
:100CB0006D0261E085E00E946D0260E086E00E94C6
:100CC0006D0265EB87E00E946D0261E085E00E94A5
:100CD0006D0261E086E00E946D0266EB87E00E9493
:100CE0006D020895FF920F931F93CF93DF938C01B2
:100CF000F62EEC0117C06D2F772785E00E946D025C
:100D00006C2F86E00E946D028F2D9927FC01EE0F5B
:100D1000FF1FE80FF91FE15FFE4F608187E00E942F
:100D20006D022196C8010596C817D90720F3E8017E
:100D30002A9617C06D2F772785E00E946D026C2FD1
:100D400086E00E946D028F2D9927FC01EE0FFF1F98
:100D5000E80FF91FE15FFE4F608187E00E946D029E
:100D60002196C8010F96C817D90720F3DF91CF91BC
:100D70001F910F91FF9008950F931F93CF93DF93CF
:100D80008C01EC010EC06D2F772785E00E946D026B
:100D90006C2F86E00E946D0260E087E00E946D0289
:100DA0002196C8010596C817D90768F3E8012A9665
:100DB0000EC06D2F772785E00E946D026C2F86E0B4
:100DC0000E946D0260E087E00E946D022196C801DA
:100DD0000F96C817D90768F3DF91CF911F910F9134
:100DE00008951F93CF93DF9380914403909145031F
:100DF00066E170E00E946C189B012E5F3F4F37FD4B
:100E00001BC0C9016AE070E00E946C18182F16958B
:100E1000C9016AE070E00E946C1887E090E0861BD0
:100E200091092EE130E0829FE001839FD00D929FD7
:100E3000D00D1124279616C0309521953F4FC9013A
:100E40006AE070E00E946C18182F16951C5FC901AB
:100E50006AE070E00E946C188EE1689FE001112446
:100E6000C950DF4F80910B0190910C01C817D90731
:100E700039F080910B0190910C010E94BC0604C0D6
:100E800080918401811721F0612FCE010E947206AA
:100E900010938401D0930C01C0930B01DF91CF918B
:100EA0001F910895AF92BF92DF92EF92FF920F933E
:100EB0001F93CF93DF93CDB7DEB721970FB6F8948A
:100EC000DEBF0FBECDBF8C01D62E5C0119826B2D0B
:100ED000772785E00E946D026A2D86E00E946D02F0
:100EE000ED2CFF24F701E35DFE4F608187E00E9457
:100EF0006D028EE190E0A80EB91E9981925E9983F1
:100F00009C3329F7F4EBAF2EB12CA00EB11E6B2D44
:100F1000772785E00E946D026A2D86E00E946D02AF
:100F2000F701E35DFE4F608187E00E946D02EEE114
:100F3000F0E0AE0EBF1EC801825F9E4FA816B90634
:100F400031F721960FB6F894DEBF0FBECDBFDF910B
:100F5000CF911F910F91FF90EF90DF90BF90AF90D6
:100F60000895EF92FF920F931F93CF93DF93CDB726
:100F7000DEB721970FB6F894DEBF0FBECDBF8C0150
:100F80007C0119826F2D772785E00E946D026E2DFE
:100F900086E00E946D0260E087E00E946D028EE1B3
:100FA00090E0E80EF91E9981925E99839C3351F787
:100FB00084EBE82EF12CE00EF11E6F2D772785E0F3
:100FC0000E946D026E2D86E00E946D0260E087E057
:100FD0000E946D02EEE1F0E0EE0EFF1EC801825F9E
:100FE0009E4FE816F90649F721960FB6F894DEBF32
:100FF0000FBECDBFDF91CF911F910F91FF90EF906A
:1010000008951F93CF93DF938091460390914703F8
:1010100066E170E00E946C189B012A5F3F4F37FD2C
:1010200012C0C9016AE070E00E946C18182F169572
:101030001C5FC9016AE070E00E946C18C6E8D0E04D
:10104000C61BD10913C0309521953F4FC9016AE0F5
:1010500070E00E946C18182F1695C9016AE070E0C4
:101060000E946C18C62FDD27C957DF4F80910D01F4
:1010700090910E01C817D90739F080910D01909118
:101080000E010E94B10704C080918501811721F0F3
:10109000612FCE010E94520710938501D0930E015B
:1010A000C0930D01DF91CF911F91089560E085E01D
:1010B0000E946D026FEC86E00E946D026CE887E092
:1010C0000E946D0261E085E00E946D026BE086E0A7
:1010D0000E946D026DE887E00E946D020895EF9214
:1010E000FF920F931F93CF93DF937A019EE1699F45
:1010F000B0011124680F711D8B01020F111D109298
:10110000A503EB0116C06D2F772785E00E946D02C5
:101110006C2F86E00E946D028091A503F701E80F15
:10112000F11D60818F5F8093A50387E00E946D02AF
:101130002196C017D10738F3DF91CF911F910F91FE
:10114000FF90EF90089525E046E051E06CE081E0EB
:101150000E946F080895CF93DF93CDB7DEB7249731
:101160000FB6F894DEBF0FBECDBF19821A8285E498
:101170008B831C82F894789430915603832F6AE015
:101180000E944C18282F0E944C18482F822F0E9432
:101190004C18292F832F0E944C18992319F48AE0A8
:1011A0008C8301C09C83222319F48AE08A8301C0C6
:1011B0002A83498324E0AE014F5F5F4F61E083E003
:1011C0000E946F0824960FB6F894DEBF0FBECDBF05
:1011D000DF91CF910895CF93DF93CDB7DEB72497FA
:1011E0000FB6F894DEBF0FBECDBF80E28A839BE0CE
:1011F000998381E38B839C8321E0AE014E5F5F4F37
:1012000061E081E00E946F0880915B01813079F498
:1012100021E0AE014F5F5F4F62E00E946F0822E065
:10122000AE014D5F5F4F63E081E00E946F0824963E
:101230000FB6F894DEBF0FBECDBFDF91CF910895FA
:1012400080915601813069F42091A301922F27FDEE
:101250009F5F959544EA51E061E08EE0891B0E9412
:101260006F080895CF93DF93CDB7DEB725970FB6FC
:10127000F894DEBF0FBECDBFDE011196EAE3F1E0C8
:1012800085E001900D928150E1F725E0AE014F5FBE
:101290005F4F67E08CE00E946F0825960FB6F894C8
:1012A000DEBF0FBECDBFDF91CF9108956CE480E02B
:1012B0000E946D0208958091580390915903843BD8
:1012C000910554F08091A003992720915603309105
:1012D00057038217930744F080918601882361F4B5
:1012E00081E080938601089580918601181614F498
:1012F0000E94560910928601089562E480E00E94DF
:101300006D020895EF92FF920F931F93CF93DF9397
:10131000CDB7DEB72F970FB6F894DEBF0FBECDBFA7
:1013200085E0FE01369611928A95E9F780914E0389
:1013300090914F036EE170E00E946C18CB018E011A
:10134000055F1F4F019797FF02C080E090E04AE0E1
:1013500050E0B8010E94E717F80101900020E9F77A
:101360003197EE2EE01A1092A503FF240AC00E0F4B
:101370001F1FEC0FFD1F83850E947904F8018083F5
:10138000F394EF2DFF278E2D992787FD90958E01E1
:101390000F5F1F4FE817F90754F3F092A50325E0FC
:1013A000AE014A5F5F4F69E085E10E946F082E2D14
:1013B000A80169E089E18E190E946F082F960FB687
:1013C000F894DEBF0FBECDBFDF91CF911F910F917B
:1013D000FF90EF900895EF92FF920F931F93CF939A
:1013E000DF93CDB7DEB72E970FB6F894DEBF0FBEF2
:1013F000CDBF19821A821B821C8280917601909146
:1014000077018E01065F1F4F4AE050E0B8010E944D
:10141000E717F80101900020E9F73197EE2EE01A66
:101420001092A503FF240AC00E0F1F1FEC0FFD1F13
:1014300082850E947904F8018083F394EF2DFF27C1
:101440008E2D992787FD90958E010B5F1F4FE81712
:10145000F90754F3F092A50324E0AE014F5F5F4F0C
:1014600066E085E10E946F082E2DA80166E089E103
:101470008E190E946F08809176019091770118165D
:10148000190664F460E085E00E946D0262EC86E07B
:101490000E946D026CE887E00E946D0280917601E7
:1014A0009091770197FF0CC060E085E00E946D028B
:1014B00062EC86E00E946D026DE887E00E946D029A
:1014C0008091760190917701892B61F460E085E04D
:1014D0000E946D0262EC86E00E946D0260E087E08F
:1014E0000E946D022E960FB6F894DEBF0FBECDBFE0
:1014F000DF91CF911F910F91FF90EF900895EF92A0
:10150000FF920F931F93CF93DF93CDB7DEB72B9747
:101510000FB6F894DEBF0FBECDBFDE011196E7E334
:10152000F1E083E001900D928150E1F78E01085FB8
:101530001F4F4AE050E0B801809154039091550349
:101540000E94E717F80101900020E9F73197EE2E8D
:10155000E01A1092A503FF240AC00E0F1F1FEC0F04
:10156000FD1F80850E947904F8018083F394EF2D9C
:10157000FF278E2D992787FD90958E010C5F1F4FB9
:10158000E817F90754F3F092A50323E0AE014F5F8B
:101590005F4F6EE08DE00E946F082E2DA8016EE077
:1015A00080E18E190E946F082B960FB6F894DEBF6B
:1015B0000FBECDBFDF91CF911F910F91FF90EF90A4
:1015C0000895EF92FF920F931F93CF93DF93CDB7C0
:1015D000DEB728970FB6F894DEBF0FBECDBF1982D5
:1015E0008AE08A8380916801909169018E010A5F87
:1015F0001F4F4AE050E0B8010E94E717F801019040
:101600000020E9F73197EE2EE01A1092A503FF248F
:101610000DC08E010D5F1F4F0E0F1F1FEC0FFD1F22
:1016200086810E947904F8018083F394EF2DFF27CF
:101630008E2D992787FD9095E817F90754F3F092BE
:10164000A50380916801909169018E010D5F1F4F84
:101650000A976CF421E0AE014F5F5F4F6CE081E0D0
:101660000E946F0821E0A8016CE082E004C022E043
:10167000A8016CE081E00E946F0880916A0190915E
:101680006B018E010A5F1F4F4AE050E0B8010E94D3
:10169000E717F80101900020E9F73197EE2EE01AE4
:1016A0001092A503FF240DC08E010D5F1F4F0E0F7A
:1016B0001F1FEC0FFD1F86810E947904F8018083B3
:1016C000F394EF2DFF278E2D992787FD9095E8172E
:1016D000F90754F3F092A50380916A0190916B0190
:1016E0008E010D5F1F4F0A976CF421E0AE014E5F33
:1016F0005F4F6CE084E00E946F0821E0A8016CE07D
:1017000085E004C022E0A8016CE084E00E946F083C
:1017100028960FB6F894DEBF0FBECDBFDF91CF91F4
:101720001F910F91FF90EF900895CF92DF92EF926B
:10173000FF920F931F93CF93DF93CDB7DEB72B9715
:101740000FB6F894DEBF0FBECDBF80915C019091C3
:101750005D0180915C0190915D018D5A964230F05F
:101760008CEA96E290935D0180935C0180915C012C
:1017700090915D0164E670E00E94581870935801E2
:101780006093570180915C0190915D0164E670E087
:101790000E94581890935A018093590180915901E1
:1017A00090915A016AE070E00E94581870935A01B3
:1017B00060935901809157019091580125E4298344
:1017C0001A821B828E01085F1F4F4AE050E0B80169
:1017D0000E94E717F80101900020E9F73197CE2E1B
:1017E000C01A1092A503DD240BC0020F131FE20ED6
:1017F000F31EF70180810E947904F8018083D3945D
:101800002D2D33278C2D992787FD909548E0E42EC8
:10181000F12CEC0EFD1E8E010C5F1F4F28173907AF
:1018200024F3D092A50322E0AE014E5F5F4F62E049
:1018300083E00E946F082C2DA80162E085E08C19DE
:101840000E946F088091590190915A014AE050E03E
:10185000B7010E94E717F70101900020E9F73197DF
:10186000EE19EE2E1092A503FF240AC00E0F1F1FC3
:10187000EC0FFD1F80850E947904F8018083F394AA
:10188000EF2DFF278E2D992787FD90958E010C5FF8
:101890001F4FE817F90754F3F092A50321E0AE01BA
:1018A0004F5F5F4F62E085E00E946F0821E0AE016C
:1018B0004E5F5F4F62E086E00E946F0821E0A80162
:1018C00062E086E00E946F082B960FB6F894DEBFA8
:1018D0000FBECDBFDF91CF911F910F91FF90EF9081
:1018E000DF90CF9008950F931F93CF93DF93CDB7E1
:1018F000DEB72A970FB6F894DEBF0FBECDBF4AE021
:1019000050E08E010F5F1F4FB8010E94E717F801EA
:1019100001900020E9F73197E01B1092A50320E029
:10192000FF27E7FDF09501C02F5F822F99278E17C3
:101930009F07D4F32093A5032A960FB6F894DEBF31
:101940000FBECDBFDF91CF911F910F9108959F9250
:10195000AF92BF92CF92DF92EF92FF920F931F93BD
:10196000CF93DF93CDB7DEB76E970FB6F894DEBF97
:101970000FBECDBF982EA62E7A01FA01019000204D
:10198000E9F73197BE2EB41ACC24DD240BC0FF2713
:101990008A010E0F1F1FEE0DFF1D80810E9479042A
:1019A000F8018083EC2D0894C11CD11C8B2D992744
:1019B0000196AE014F5F5F4FC816D90641F72B2D38
:1019C0006A2D892D0E946F086E960FB6F894DEBFBF
:1019D0000FBECDBFDF91CF911F910F91FF90EF9080
:1019E000DF90CF90BF90AF909F900895EF92FF92BD
:1019F0000F931F93CF93DF93CDB7DEB764970FB6E6
:101A0000F894DEBF0FBECDBFE82EF62ECA014AE025
:101A100050E08E010F5F1F4FB8010E94E717A80129
:101A20006F2D8E2D0E94A70C64960FB6F894DEBF22
:101A30000FBECDBFDF91CF911F910F91FF90EF901F
:101A4000089560915E0170915F01809160019091B5
:101A5000610128E631E040E050E00E947F18A901D2
:101A600063E083E00E94F60C0895BF92CF92DF926C
:101A7000EF92FF920F931F93CF93DF93CDB7DEB713
:101A800064970FB6F894DEBF0FBECDBFB82EC62E3A
:101A90009A01DE01119605C0EA0FFB1F90832F5FAC
:101AA0003F4F822F841BF9019491E82FFF27992340
:101AB00099F7EA0FFB1F1082FD0101900020E9F762
:101AC0003197DE2EDA1AEE24FF2409C08D01020FB1
:101AD000111DF80180810E947904F80180832E2D68
:101AE0000894E11CF11C8D2D99270196DE011196B9
:101AF000E816F90659F72D2DAD016C2D8B2D0E949E
:101B00006F0864960FB6F894DEBF0FBECDBFDF91AD
:101B1000CF911F910F91FF90EF90DF90CF90BF90EA
:101B20000895EF92FF920F931F93CF93DF9333E0CB
:101B3000E32EF12CC0E0D0E0AFEAB2E08C91FD01E1
:101B4000218112810381B7016C5F7F4F7B01149665
:101B5000F2E0633D7F0709F456C0422F55274D53ED
:101B60005040E0914301F0914401EC0FFD1F992793
:101B7000CD97880F991F880F991F9A01689413F8C1
:101B8000359527951694E1F7822B932B8083673246
:101B90007105C9F1212F33272D533040FE013196B5
:101BA0008091430190914401E80FF91F4F705070EC
:101BB00084E0440F551F8A95E1F7C90195958795F3
:101BC00095958795482B592B408381E06B37780793
:101BD000D1F0FE0132968091430190914401E80FCB
:101BE000F91F2370307086E0220F331F8A95E1F7CA
:101BF000802F9927CD97282B392B20836F5C72403B
:101C000011F023969BCFDF91CF911F910F91FF9001
:101C1000EF900895AF92BF92CF92DF92EF92FF9232
:101C20000F931F93CF93DF938091BA01843409F00F
:101C300074C003E010E060E070E092E0C92ED12CA7
:101C400081E0E82EF12CCBEBD1E088812981BA80AC
:101C5000AB800C5F1F4F24966134710519F4A1E429
:101C6000B0E05FC0422F55274D535040E0914101F5
:101C7000F0914201E60FF71F9927CD97880F991F22
:101C8000880F991F9A01A4E035952795AA95E1F749
:101C9000822B932B8083D7016034710509F441C0F6
:101CA0002B2D33272D5330408091410190914201DB
:101CB000A80FB91F4F705070F4E0440F551FFA95EC
:101CC000E1F7C9019595879595958795482B592BEF
:101CD0004C93D6010B35110521F180914101909172
:101CE0004201A80FB91F2370307046E0220F331F46
:101CF0004A95E1F78A2D9927CD97282B392B2C93DC
:101D0000DB01139683E090E0C80ED91EE80EF91EA1
:101D1000A134B10531F0BD0198CF03E010E0A0E09F
:101D2000B0E08091BA01813509F067C068E170E0E8
:101D3000E801C854DE4F888129811A810B812496DD
:101D40006115710509F459C0422F55274D53504074
:101D5000E0914501F0914601EA0FFB1F9927CD97CD
:101D6000880F991F880F991F9A01689413F8359569
:101D700027951694E1F7822B932B808361307105B0
:101D8000E1F1212F33272D533040FD013196809111
:101D9000450190914601E80FF91F4F70507084E0A3
:101DA000440F551F8A95E1F7C9019595879595953B
:101DB0008795482B592B4083AB0143505040BA01C3
:101DC0009FEF4F3F5907C9F0FD01329680914501C1
:101DD00090914601E80FF91F2370307016E0220F32
:101DE000331F1A95E1F7802F9927CD97282B392B90
:101DF0002083452B11F013969ECF10925401DF9152
:101E0000CF911F910F91FF90EF90DF90CF90BF90F7
:101E1000AF900895EF92FF920F931F93CF93DF93AC
:101E20008091AE02843409F091C033E0E32EF12CAE
:101E300060E070E0AFEAB2E08C91FD012181128197
:101E40000381E70124967E0114966134710509F43B
:101E500056C0422F55274D535040E0913F01F0911D
:101E60004001E60FF71F9927CD97880F991F880F1C
:101E7000991F9A01689413F8359527951694E1F700
:101E8000822B932B808360347105C9F1212F332776
:101E90002D533040FB01319680913F0190914001DC
:101EA000E80FF91F4F70507084E0440F551F8A955A
:101EB000E1F7C9019595879595958795482B592BFD
:101EC0004083CB35D105D9F0FB01329680913F019B
:101ED00090914001E80FF91F2370307046E0220F07
:101EE000331F4A95E1F7802F9927CD97282B392B5F
:101EF00020836E33710519F06D5F7F4F9DCF809108
:101F0000580390915903843B91058CF480916201B0
:101F10008130E1F410926201F8940E940A107894E2
:101F20008091580390915903843B91057CF08091F6
:101F30006201882359F481E080936201F8948091D2
:101F40005501882311F40E94FA0F78948091AE0213
:101F50008C3459F481E090E090937F0180937E016E
:101F600081E0809381010E94910D8091AE028D34B9
:101F700059F482E090E090937F0180937E0181E0AC
:101F8000809381010E94910D8091AE028E3459F4AC
:101F900083E090E090937F0180937E0181E08093C5
:101FA00081010E94910D8091AE028F3459F484E03A
:101FB00090E090937F0180937E0181E08093810186
:101FC0000E94910D8091AE02803559F485E090E039
:101FD00090937F0180937E0181E0809381010E9434
:101FE000910D10925301DF91CF911F910F91FF90AE
:101FF000EF90089582E289B910BC80B91CBE909A16
:1020000028E92AB996E890BD82EC8BB921B99CBF2A
:1020100082B9089582E289B910BC80B91CBE909A39
:1020200088E98AB926E820BD92EC9BB980E981B99C
:102030002CBF92B90895159BFECF83B908951F92C6
:102040000F920FB60F9211248F939F93EF93FF93EC
:102050009CB19093A6039D30A1F4809188018130BA
:1020600081F4AB981092880180935401E09187032A
:10207000FF27E854FE4F908380918703809390025E
:102080002CC080918801882319F0813031F513C06C
:10209000933239F480915401882319F481E08093BC
:1020A00088011092870380918703E82FFF27E85467
:1020B000FE4F90830CC0E0918703FF27E854FE4F4A
:1020C000908380918703853930F4809187038F5FF7
:1020D0008093870302C010928801FF91EF919F9136
:1020E0008F910F900FBE0F901F9018951F920F9217
:1020F0000FB60F9211248F939F93EF93FF9393B199
:102100009093A7039D3081F480918701813061F421
:10211000AB981092870180935301E0918403FF27CD
:10212000E455FD4F90832DC080918701882319F0DD
:10213000813039F514C0933241F4809153018823E2
:1021400021F481E080938701AB9A109284038091FF
:102150008403E82FFF27E455FD4F90830CC0E091E6
:102160008403FF27E455FD4F9083809184038539D4
:1021700030F4809184038F5F8093840302C01092B7
:102180008701FF91EF919F918F910F900FBE0F905C
:102190001F901895CF93DF93CDB7DEB72C970FB66E
:1021A000F894DEBF0FBECDBF83E289831A8281E738
:1021B0008B838CE78C838DE68D838DE38E838F8379
:1021C00020E030E0FE013196AE01485F5F4F819123
:1021D000280F311DE417F507D1F7C90160E070E160
:1021E0000E946C189C0160E470E00E946C18635CB3
:1021F0006887C90160E470E00E946C18835C89877D
:102200008DE08A87FE0131969E01255F3F4F8081D8
:10221000159BFECF83B93196E217F307C1F72C96D1
:102220000FB6F894DEBF0FBECDBFDF91CF910895FA
:10223000CF93DF93CDB7DEB72A970FB6F894DEBF02
:102240000FBECDBF83E289831A8283E68B831C8213
:102250001D8286E890E060E070E10E946C189C01AD
:1022600060E470E00E946C18635C6E83C90160E4F6
:1022700070E00E946C18835C8F838DE08887FE017C
:1022800031969E01275F3F4F8081159BFECF83B91A
:102290003196E217F307C1F72A960FB6F894DEBF1E
:1022A0000FBECDBFDF91CF91089585B392E089270E
:1022B00085BB089590916501913019F485B3892704
:1022C00085BB08951F920F920FB60F9211242F9382
:1022D0003F935F936F937F938F939F93AF93BF933E
:1022E0008091890190918A01892B81F484B595B5FB
:1022F0009093900180938F018EB58F7B8EBD81E08E
:1023000090E090938A018093890141C084B595B58E
:1023100090938E0180938D012EB520642EBD209167
:102320008F0130919001821B930B10928A011092C1
:102330008901865698406CE271E00E9458187093AB
:102340008C0160938B0177FF05C010928C01109275
:102350008B0109C06730710534F086E090E09093FE
:102360008C0180938B0120918B0130918C018091A5
:102370000201992787FD90952817390741F02630EB
:1023800031052CF42093020181E080936C01BF9110
:10239000AF919F918F917F916F915F913F912F911D
:1023A0000F900FBE0F901F90189580914E03909143
:1023B0004F0390936F0180936E0180916E01909115
:1023C0006F012091700130917101821B930B9093EA
:1023D00073018093720180916E0190916F019093CF
:1023E00071018093700140917A0150917B0120919D
:1023F000720130917301CA01E3E0880F991FEA95D9
:10240000E1F7841B950B73E0220F331F7A95E1F7F8
:10241000820F931F68E070E00E946C1870937B013C
:1024200060937A0120917C0130917D0140917A0185
:1024300050917B01C90163E0880F991F6A95E1F70C
:10244000821B930B840F951F68E070E00E946C184C
:1024500070937D0160937C0180917C0190917D015E
:1024600090937701809376010E94EB090895BF92C3
:10247000CF92DF92EF92FF920F931F93CF93DF9350
:10248000CDB7DEB760970FB6F894DEBF0FBECDBFF5
:1024900019821A821B821C82809186029091870287
:1024A0009093AB038093AA03809188029091890254
:1024B0009093A9038093A8038091AA039091AB0302
:1024C0008E01055F1F4F4AE050E0B8010E94E717F8
:1024D000F80101900020E9F73197BE2EB01ACC2404
:1024E000DD240DC0EC0CFD1CF70180810E947904F5
:1024F0000C0D1D1DF80180830894C11CD11C8B2D6F
:10250000992787FD90952BE0E22EF12CEC0EFD1E15
:102510008E010B5F1F4FC816D90624F324E0AE01CD
:102520004F5F5F4F61E08CE00E946F082B2DA80188
:1025300061E080E18B190E946F088091A80390915F
:10254000A9034AE050E0B7010E94E717F7010190A4
:102550000020E9F73197DE2EDE18EE24FF240DC0AF
:10256000FE01EE0DFF1D83850E9479040E0D1F1DD7
:10257000F80180830894E11CF11C8D2D992787FDBB
:1025800090958E010B5F1F4FE816F9064CF324E07F
:10259000AE014F5F5F4F62E08CE00E946F082D2D0F
:1025A000A80162E080E18D190E946F0860960FB665
:1025B000F894DEBF0FBECDBFDF91CF911F910F9179
:1025C000FF90EF90DF90CF90BF900895DF92EF9251
:1025D000FF920F931F93CF93DF93CDB7DEB72B9767
:1025E0000FB6F894DEBF0FBECDBFDE011196EBE44F
:1025F000F1E083E001900D928150E1F78E01085FD8
:102600001F4F8091AB024AE050E0B80199270E9429
:10261000E717F80101900020E9F73197DE2ED01A74
:10262000EE24FF240DC0FE01EE0DFF1D80850E94EB
:1026300079040E0D1F1DF80180830894E11CF11C24
:102640008D2D992787FD90958E010C5F1F4FE81601
:10265000F9064CF323E0AE014F5F5F4F61E088E184
:102660000E946F082D2DA80161E08BE18D190E9459
:102670006F082B960FB6F894DEBF0FBECDBFDF916B
:10268000CF911F910F91FF90EF90DF90089522E07E
:1026900049E451E061E08AE10E946F0808956F9279
:1026A0007F928F929F92BF92CF92DF92EF92FF9292
:1026B0000F931F93CF93DF93CDB7DEB764970FB619
:1026C000F894DEBF0FBECDBF19821A821B821C8216
:1026D0006090A7027090A8028090A9029090AA0230
:1026E0008E01035F1F4F6091A3027091A40280913D
:1026F000A5029091A6022AE030E0A8010E940818E5
:10270000F80101900020E9F73197BE2EB01ACC24D1
:10271000DD240DC0EC0CFD1CF70180810E947904C2
:102720000C0D1D1DF80180830894C11CD11C8B2D3C
:10273000992787FD90953DE0E32EF12CEC0EFD1ED0
:102740008E010B5F1F4FC816D90624F324E0AE019B
:102750004F5F5F4F6DE084E10E946F082B2DA80151
:102760006DE088E18B190E946F082AE030E0A70134
:10277000C401B3010E940818F70101900020E9F795
:102780003197DE2EDE18EE24FF240DC0FE01EE0D83
:10279000FF1D85850E9479040E0D1F1DF8018083A1
:1027A0000894E11CF11C8D2D992787FD90958E01D1
:1027B0000B5F1F4FE816F9064CF324E0AE014F5FA4
:1027C0005F4F6EE084E10E946F082D2DA8016EE03E
:1027D00088E18D190E946F0864960FB6F894DEBFE9
:1027E0000FBECDBFDF91CF911F910F91FF90EF9062
:1027F000DF90CF90BF909F908F907F906F900895C3
:10280000F89488E190E028E00FB6F894A89581BD8F
:102810000FBE21BDFFCF1F939D9902C180919101F1
:102820008F5F8093910191E090939301809191014A
:10283000853009F0F9C080919501882309F071C0B5
:10284000909395011092960164E084E00E946D02DD
:102850002091A30144EA51E061E083E00E946F0807
:1028600041E951E063E083E00E94350D68E084E0D7
:102870000E946D024AE951E065E083E00E94350D57
:1028800080910001813019F44DEB51E002C040EC21
:1028900051E065E084E10E94350D60E084E00E9433
:1028A0006D024EE951E066E083E00E94350D8091B3
:1028B0005501813019F44DEB51E002C040EC51E07C
:1028C00066E084E10E94350D44EA51E067E083E070
:1028D0000E94350D80915601813019F44DEB51E085
:1028E00002C040EC51E067E084E10E94350D4CEA03
:1028F00051E068E083E00E94350D80916D018130E8
:1029000019F44DEB51E002C040EC51E068E084E185
:102910000E94350D48EB51E06BE083E00E94350DDD
:1029200081C010919601113001F568E084E00E94A9
:102930006D0280915501882329F4109355014DEBC8
:1029400051E004C01092550140EC51E066E084E192
:102950000E94350D80915501A0E0B0E0082E0E9444
:10296000A91860E084E00E946D0280919601823097
:1029700009F568E084E00E946D0280915601882389
:1029800031F481E0809356014DEB51E004C0109288
:10299000560140EC51E067E084E10E94350D8091E2
:1029A0005601A2E0B0E0082E0E94A91860E084E081
:1029B0000E946D0280919601833009F568E084E001
:1029C0000E946D0280916D01882331F481E0809333
:1029D0006D014DEB51E004C010926D0140EC51E0EF
:1029E00068E084E10E94350D80916D01A7E1B0E0BF
:1029F000082E0E94A91860E084E00E946D02809178
:102A00009601843089F410929501F89488E190E061
:102A100028E00FB6F894A89581BD0FBE21BDFFCF69
:102A200010929101109293019C99E9C090919501A7
:102A3000913009F0EAC090939401809192018F5FE8
:102A40008093920180919201853009F0DEC010924E
:102A5000920180919601823009F464C0833030F491
:102A6000882359F0813009F0D0C031C0833009F497
:102A700083C0843009F0C9C09EC0909396014AE992
:102A800051E065E083E00E94350D809100018130C6
:102A900019F44DEB51E002C040EC51E065E084E1F7
:102AA0000E94350D68E084E00E946D024EE951E01D
:102AB00066E083E00E94350D80915501813019F464
:102AC0004DEB51E002C040EC51E066E090C082E086
:102AD000809396014EE951E066E083E00E94350D57
:102AE00080915501813019F44DEB51E002C040EC6A
:102AF00051E066E084E10E94350D68E084E00E94C8
:102B00006D0244EA51E067E083E00E94350D809158
:102B10005601813019F44DEB51E002C040EC51E018
:102B200067E065C083E08093960144EA51E067E086
:102B30000E94350D80915601813019F44DEB51E022
:102B400002C040EC51E067E084E10E94350D68E08E
:102B500084E00E946D024CEA51E068E083E00E944C
:102B6000350D80916D01813019F44DEB51E002C0BB
:102B700040EC51E068E03BC084E0809396014CEA71
:102B800051E068E083E00E94350D80916D01813055
:102B900019F44DEB51E002C040EC51E068E084E1F3
:102BA0000E94350D68E084E00E946D0248EB51E020
:102BB0006BE083E01DC01092960148EB51E06BE0A2
:102BC00083E00E94350D68E084E00E946D024AE9CE
:102BD00051E065E083E00E94350D80910001813075
:102BE00019F44DEB51E002C040EC51E065E084E1A6
:102BF0000E94350D60E084E00E946D0206C01092D4
:102C0000920180919301809194011F9108958130E8
:102C100029F4A0E0B0E0062E0E94A9180895EF92D2
:102C2000FF920F931F93CF93DF93CDB7DEB76497D7
:102C30000FB6F894DEBF0FBECDBF40E050E08E016E
:102C40000F5F1F4F842F9927DC01AD5FBF4F0E949C
:102C5000A118202D3327F801E80FF91F2083222324
:102C6000F1F04F5F5F4F2F3F69F7108218C0FE01F0
:102C7000E00FF11F81810E9479040C551E4FF8016D
:102C800080830E2D11270894E11CF11C8091A30173
:102C9000992787FD9095081719074CF30EC0DE01A0
:102CA0001196FD0101900020E9F73197EA1BFB0B1B
:102CB000E093A301EE24FF24E4CF64960FB6F894CA
:102CC000DEBF0FBECDBFDF91CF911F910F91FF905F
:102CD000EF9008951F920F920FB60F9211248F93C9
:102CE0009F9380919A018130A1F0813018F0823059
:102CF00049F525C0809198018E3129F410929801F0
:102D000081E080939A01809198018F5F8093980170
:102D100019C090919901923061F4109299018091BB
:102D20009701813019F490939A0103C083E0809356
:102D30009A01809199018F5F8093990103C083E08C
:102D400080939A019F918F910F900FBE0F901F90CB
:102D500018951F920F920FB60F9211248F938091A6
:102D60009A01833011F410929A018F910F900FBE47
:102D70000F901F901895809144039091450365E052
:102D800070E00E946C1866507F4F77FD0FC081E0A5
:102D9000653F78071CF064EF71E003C06B3F71057D
:102DA0003CF06A5F81E08093970104C060E070E0CE
:102DB0001092970162BD08951F920F920FB60F9265
:102DC0001124EF92FF920F931F932F933F934F93F2
:102DD0005F936F937F938F939F93AF93BF93EF9383
:102DE000FF9380919B01882389F4809180009091CA
:102DF00081009093A2018093A10180918A008F7B32
:102E000080938A0081E080939B017FC08091800045
:102E10009091810090935D0180935C0180918A0084
:102E2000806480938A00109289001092880010922A
:102E30009B0180915C0190915D012091A1013091F5
:102E4000A201821B930B90935D0180935C018091A2
:102E50005C0190915D019695879590935D018093BB
:102E60005C0180915C0190915D018456904090934B
:102E70005D0180935C0180915C0190915D019C01FA
:102E80004427552780919C0190919D01A0919E011E
:102E9000B0919F01280F391F4A1F5B1F20939C018F
:102EA00030939D0140939E0150939F018091A0011A
:102EB000843130F11092A001E0905E01F0905F014A
:102EC0000091600110916101CA01B90124E130E073
:102ED00040E050E00E947F18E20EF31E041F151F11
:102EE000E0925E01F0925F01009360011093610136
:102EF00010929C0110929D0110929E0110929F01D0
:102F00008091A0018F5F8093A001FF91EF91BF910D
:102F1000AF919F918F917F916F915F914F913F9171
:102F20002F911F910F91FF90EF900F900FBE0F9078
:102F30001F901895CF93DF93CDB7DEB760970FB68C
:102F4000F894DEBF0FBECDBF80915403909155031E
:102F500090939202809391028091910290919202BB
:102F60006FE070E00E945818AE014B5F5F4FDA01CE
:102F7000641BCE014096E62FEA0FFF27ED53FE4F6C
:102F8000E491ED93A817B907B1F719821A821B8251
:102F90001C822BE06CE089E00E946F0824E0AE0107
:102FA0004F5F5F4F6BE08EE00E946F08409191028F
:102FB000509192026BE08FE00E94F60C60960FB683
:102FC000F894DEBF0FBECDBFDF91CF910895FB0116
:102FD0009F01E8944230C4F04532B4F44A3029F4F9
:102FE00097FB1EF4909581959F4F642F77270E9441
:102FF0005818805D8A330CF0895D8193CB0100976E
:10300000A1F716F45DE251931082C9010C943C18AB
:10301000FA01CF93FF93EF93223044F1253234F538
:10302000C22FE894CA3049F497FB3EF490958095FE
:10303000709561957F4F8F4F9F4F2C2F33274427DB
:103040005527FF93EF930E947F18EF91FF91605DEA
:103050006A330CF0695D6193B901CA016050704038
:103060008040904051F716F4CDE2C19310828F91C9
:103070009F91CF910C943C18DC01FC010190002041
:10308000E9F73297AE17BF0730F47C916081708307
:1030900031976D93F7CF0895991B79E004C0991F7C
:1030A000961708F0961B881F7A95C9F780950895A2
:1030B000AA1BBB1B51E107C0AA1FBB1FA617B7075E
:1030C00010F0A61BB70B881F991F5A95A9F780957A
:1030D0009095BC01CD01089597FB092E07260AD0D3
:1030E00077FD04D0E5DF06D000201AF470956195D5
:1030F0007F4F0895F6F7909581959F4F0895A1E22F
:103100001A2EAA1BBB1BFD010DC0AA1FBB1FEE1F61
:10311000FF1FA217B307E407F50720F0A21BB30BAC
:10312000E40BF50B661F771F881F991F1A9469F728
:1031300060957095809590959B01AC01BD01CF0184
:103140000895E199FECFBFBBAEBBE09A11960DB2D8
:103150000895E199FECFBFBBAEBB0DBA11960FB675
:0A316000F894E29AE19A0FBE089578
:10316A0001010300000A0000440000230023005468
:10317A00646653636552620051610050600050609A
:10318A00005161005262005363655464666768695E
:10319A006A6B6B6A69686700000053536353534252
:0E31AA00034E02880393020D0A0A1D00000066
:00000001FF
